:1000000000308A006F290000831A0A28A500030E19
:10001000A6000F288312A500030EA600A6140A0846
:10002000AD008A01A50E0408A7002008A800210839
:10003000A9002208AA002308AB002408AC00831200
:100040008B1E24280B19B8288C308400801D2A2888
:100050008C195728270884002808A0002908A10027
:100060002A08A2002B08A3002C08A400260E830057
:100070008312250EA618831609000A108A100A1189
:100080008207FC346034DA34F2346634B634BE3479
:10009000E034FE34F6340A108A100A11820738342C
:1000A0002E3438342E3438342E34383400348C1115
:1000B000831614088312C2002530C205C2154208F7
:1000C000A0000930200203197628293020020319E4
:1000D00080280C30200203199E282C30200203199E
:1000E0009E28283020020319B328B4288316141838
:1000F0007B288312762883121308C300B201B62826
:100100008316141885288312802883121308C300CD
:10011000B208031D8F2801304302AE009C28B208AC
:1001200003199C28AE0A0130AE052F302E0784003B
:10013000430880000230B100B20AB628AE0A01308E
:10014000AE052F302E0784000008C4004408930039
:1001500014168C118316141CAF288312AA280130A0
:100160008312B100B628B6288A0100288A112A28ED
:10017000FF3086000510381805148510B81885144E
:1001800033303807840000088600B8030330B80510
:100190000B118A112A28B701FF30B300FF30B400D9
:1001A000FF30B500FF30B600FF3086000034A030CD
:1001B000831693008C158312831686010510851013
:1001C0008312CB208629BA018316071487140715DA
:1001D000831207183A148718BA1407193A153A08FF
:1001E000A1009C29F0308316930583123B08073940
:1001F000A0000310A00D2008831693048312A029E9
:100200003B080D3C031D0629B70150293708BC00E7
:100210003B082E3C031D1029BC030330BC051329E9
:10022000B70A0330B7053C08BD003B08BE003E08D6
:100230002E3C031D222933303D0784000008FE397F
:10024000800050293E08203C031D2829BF014A296F
:100250003E082D3C031D2F290230BF004A293E08CD
:10026000453C031D36299E30BF004A293E08723C9A
:10027000031D3D290A30BF004A293030BE023E0826
:10028000093C031C48293E083D20A100BF004A2923
:100290009230BF0033303D0784003F088000800962
:1002A00000343A3084000008031965290130A100A8
:1002B000A001A00B5929A10B58294A30A000A00B7E
:1002C0005F2900000000800B56290034B701D629B1
:1002D000141F6E2914131308BA008C11DB29840132
:1002E0001F308305073083169F0087150716A0303F
:1002F0009300363083129400AE01B101B201B30114
:10030000B401B501B601B701B801D728A001A01DFD
:10031000912907308101813084000008C0390F38ED
:1003200080006400813084000008C039200480000F
:100330008B16C0308B04E3282108BA00BB00F228DA
:100340009412BA013A084B20BA0ABB0000210730C8
:100350003A02031DA229FA30B900B9080319B629D7
:100360000230BA0051216400B903AD29CB20FA3024
:10037000B900B9080319C2290230BA00512164003A
:10038000B903B929941664003108023C031DDA2927
:10039000B101AE08031DDA292F08B900B908031D01
:1003A000D329CB20DA29390BD7296629DA2939084C
:0A03B000BB0000216829C329630087
:02400E00763DFD
:00000001FF
